:10F000004BC0000080C000007EC000007CC000003B
:10F010007AC0000078C0000076C0000074C0000014
:10F0200072C0000070C000000BC500006CC0000082
:10F030006AC0000068C0000066C0000064C0000034
:10F0400062C0000060C000005EC000005CC0000044
:10F05000FDC2000058C0000056C0000054C00000AF
:10F0600052C0000050C000004EC000004CC0000064
:10F070004AC0000048C0000046C0000044C0000074
:10F0800042C0000040C000003EC000003CC0000084
:10F090003AC0000038C0000011241FBECFEFD0E1FD
:10F0A000DEBFCDBF04B603FE19C08091A0019091D0
:10F0B000A10182349C4D91F484B7877F84BF88E19D
:10F0C0000FB6F89480936000109260000FBE10920B
:10F0D000A1011092A001E0E0F0E0099511E0A0E0AC
:10F0E000B1E0E2E1FEEF02C005900D92A239B10756
:10F0F000D9F721E0A2E9B1E001C01D92A03AB20720
:10F10000E1F731D084C67CCF84E08093E900809120
:10F11000E80085FD0EC08091E8008B778093E800C1
:10F120008091E80082FDF3CF8EB38111F9CF80E0AA
:10F1300008958091F100089593E09093E9009091F3
:10F14000E80095FF03C08093F10008959091E800D6
:10F150009E779093E8009091E80090FDF4CF9EB3E5
:10F160009111F9CF0895CF93DF9300D01F92CDB7BF
:10F17000DEB784B7877F84BF88E10FB6F8948093A9
:10F180006000109260000FBE90E080E80FB6F89427
:10F1900080936100909361000FBE11E015BF82E083
:10F1A00085BF33D410936F0083E0809381007894FF
:10F1B000A3E07A2EB5E06B2E212C312C809100013A
:10F1C000882309F42CC284E08093E9008091E80050
:10F1D00082FF23C299DF982F853419F41092000121
:10F1E00007C088E8890F823010F0943521F48CDF55
:10F1F0008DE0A2DFEAC19035D9F39C34C9F394378E
:10F2000011F484E47BC0913611F489E5F2CF913496
:10F2100091F47ADF082F78DF90E0880F991F202F74
:10F2200030E0322F2227330F822B932BAA2797FD12
:10F23000A095BA2F9EC1903711F483E5DACF9335AC
:10F2400071F47AE8E72E71E0F72EF70181917F01E2
:10F2500073DFF1E9EF16F1E0FF06B9F7B6C19635B5
:10F2600021F481E369DF80E3C4CF933731F482E88E
:10F2700063DF86E961DF8EE1BCCF9536A1F4E0E083
:10F28000F0E070925700E89507B600FCFDCF609261
:10F290005700E89507B600FCFDCFF395E11580EF28
:10F2A000F80779F7A5CF9C3651F42EDF809599E0C9
:10F2B000E1E0F0E0082E90935700E89599CF92375F
:10F2C00021F489E0E1E0F0E010C0963419F489E01F
:10F2D000F1010BC09E3421F489E0E3E0F0E005C0C9
:10F2E000913539F489E0E2E0F0E0809357008491B1
:10F2F00080CF923631F489E51FDF81E01DDF80E0A9
:10F3000078CF923419F0973609F0CEC09983FCDE9D
:10F31000A82EB12CBA2CAA24F7DEA82AF5DE082FD5
:10F320008BEB800F9981823010F08FE362CF97369C
:10F3300009F044C081E180935700E8954501B12C64
:10F340008114910409F441C1C0909201D0909301BD
:10F35000E0909401F09095010634B9F4EB2DF0E0C3
:10F36000EC29FD298491E8DEBB2069F0F2E0CF0EA4
:10F37000D11CE11CF11CC0929201D0929301E09249
:10F380009401F0929501B12615C0D701C601B6953A
:10F39000A7959795879525D5CFDE82E0C80ED11C1D
:10F3A000E11CF11CC0929201D0929301E092940171
:10F3B000F092950191E0891A9108C2CFC090920114
:10F3C000D0909301E0909401F0909501063429F0DB
:10F3D000BB82AA82412C512C31C0F6017092570099
:10F3E000E89507B600FCFDCFF3CF063479F555203C
:10F3F00051F18090920190909301A0909401B0906F
:10F40000950182DE242D30E0382BF40109011093A0
:10F410005700E8951124F2E08F0E911CA11CB11C3D
:10F420008092920190929301A0929401B0929501E2
:10F4300051268A819B8101979B838A83EA81FB8184
:10F44000EF2B99F626C060DE482EF2CF5DDE682FE6
:10F450008091920190919301A0919401B0919501B6
:10F46000B695A79597958795C4D480919201909170
:10F470009301A0919401B09195010296A11DB11D37
:10F480008093920190939301A0939401B09395017E
:10F49000D0CF063409F0ACCEF60160925700E89563
:10F4A00007B600FCFDCFA4CE933469F4E09092013E
:10F4B000F090930129DE90E0F7010C0110935700C2
:10F4C000E895112495CE9336F9F4C0909201D0902E
:10F4D0009301E0909401F090950116DEF601E16051
:10F4E00090E00C0110935700E8951124F2E0CF0E44
:10F4F000D11CE11CF11CC0929201D0929301E092C8
:10F500009401F092950174CE9D3659F4E0919201E8
:10F51000F091930160925700E89507B600FCFDCF8B
:10F5200067CE923551F4E0919201F0919301E5900C
:10F53000F4908F2D01DE8E2D5CCE943419F5E4DD30
:10F54000682F8091920190919301A0919401B091C4
:10F550009501B695A795979587954BD48091920183
:10F5600090919301A0919401B09195010296A11DF3
:10F57000B11D8093920190939301A0939401B09355
:10F58000950136CE9436F1F4C0909201D09093015B
:10F59000E0909401F0909501D701C601B695A7952A
:10F5A000979587951ED4C8DD82E0C80ED11CE11C5A
:10F5B000F11CC0929201D0929301E0929401F092DA
:10F5C000950103C09B3109F0B0CE7092E900909193
:10F5D000E8008091E8008E778093E80095FD11C0E7
:10F5E0008091E80080FD04C08EB38111F9CF15C071
:10F5F0008091E8008E778093E80003C08EB3882363
:10F6000061F08091E80080FFF9CF94E09093E900E9
:10F610008091E8008B778093E800C8D3CFCD8091AC
:10F62000E00081608093E00082E49CED9093A10172
:10F630008093A0012CE088E190E00FB6F894A895A3
:10F64000809360000FBE20936000FFCF1F920F9247
:10F650000FB60F9211240F900FBE0F901F901895A8
:10F6600042E061EC82E05ED142E161E883E05AD1A0
:10F6700042E160E884E056C180919801982F9F771D
:10F68000913299F590919901913229F0923229F1B4
:10F69000903259F510C0813A41F58091E800877F9A
:10F6A0008093E80067E070E081E091E0A4D0809171
:10F6B000E8008B770FC08132C1F48091E800877F2A
:10F6C0008093E80067E070E081E091E0EFD0809106
:10F6D000E8008E778093E8000895813231F48091BC
:10F6E000E800877F8093E80031C10895292F30E03A
:10F6F0002230310539F02330310549F02130310510
:10F7000061F410C08EE390E02AE331E01EC088234C
:10F7100071F0813089F08230A1F080E090E020E04B
:10F7200030E013C082E190E028E731E00EC084E0D1
:10F7300090E026E331E009C088E190E02CE131E07F
:10F7400004C082E190E028E031E0FA0131832083B7
:10F75000089507B600FCFDCFF999FECF23E0FB0129
:10F7600020935700E89507B600FCFDCF81E1809318
:10F770005700E895089507B600FCFDCFF999FECF34
:10F7800025E0FB0120935700E89507B600FCFDCF6C
:10F7900081E180935700E895089507B600FCFDCFFE
:10F7A000F999FECF21E0FB010A0120935700E8956B
:10F7B0001124089521E2FC012093570084910895BB
:10F7C00029E0FC012093570084910895E1E0F0E0E6
:10F7D00089E0809357008491089507B600FCFDCF1F
:10F7E000F999FECF809599E0E1E0F0E0082E909342
:10F7F0005700E895089520919E0130919F012617AA
:10F80000370748F06115710539F42091E8002E772B
:10F810002093E80001C0B901FC0120E061157105E9
:10F8200091F18EB38823E1F18530E1F18091E80018
:10F8300083FD3AC08091E80082FF06C08091E80015
:10F8400082FF24C080E008958091E80080FFE6CF29
:10F850008091F2009091F3006115710551F08830AC
:10F86000910538F421912093F100615071090196BE
:10F87000F3CF21E0089709F020E08091E8008E772F
:10F880008093E800CBCF2111CCCFD8CF8EB3882383
:10F8900039F0853039F08091E80083FFCFCF04C084
:10F8A00082E0089583E0089581E00895611571056F
:10F8B00029F42091E8002B772093E8006115710569
:10F8C00021F12EB3222351F1253051F12091E8008E
:10F8D00023FD20C02091E80022FFF3CFFC01CF01DF
:10F8E0002091F2003091F300232B19F38091F10065
:10F8F0008193CF01615071096115710581F7D9CFED
:10F900008EB3882359F0853059F08091E80080FF4C
:10F91000F7CF02C081E0089580E0089582E0089565
:10F9200083E008958F708093E900EBEEF0E0808132
:10F9300081608083EDEEF0E010826093EC00408304
:10F940008091EE00881F8827881F08958091980174
:10F9500087FD05C08091E80080FF0DC010C0809138
:10F96000E80082FD04C08EB38111F9CF0895809123
:10F97000E8008B7707C08EB38111ECCF089580919A
:10F98000E8008E778093E80008950F931F93CF933C
:10F99000DF9349D050D0C8EDD0E088818F7788833D
:10F9A00088818068888388818F7D8883E7EDF0E097
:10F9B00080818068808319BC1EBA1092960100EE87
:10F9C00010E0F80180818B7F80838881816088834B
:10F9D00042E060E080E0A6DFE1EEF0E080818E7F33
:10F9E0008083E2EEF0E080818160808380818860A6
:10F9F0008083F80180818E7F808388818061888305
:10FA0000DF91CF911F910F910895E8EDF0E0808193
:10FA10008F7E8083E7EDF0E080818160808381E0EC
:10FA200080939701B2CFE8EDF0E080818C7F8083F6
:10FA30001092E20008951092DA001092E100089509
:10FA40001F920F920FB60F9211242F933F934F9353
:10FA50005F936F937F938F939F93AF93BF93EF9336
:10FA6000FF938091DA0080FF1BC08091D80080FF57
:10FA700017C08091DA008E7F8093DA008091D900E0
:10FA800080FF0BC08CE089BD8EE089BD09B400FE0B
:10FA9000FDCF81E08EBB89D103C019BC1EBA85D1D0
:10FAA0008091E10080FF17C08091E20080FF13C0C9
:10FAB0008091E2008E7F8093E2008091E20080617D
:10FAC0008093E2008091D80080628093D80019BCB6
:10FAD00085E08EBB6AD18091E10084FF2EC08091C9
:10FAE000E20084FF2AC08CE089BD8EE089BD09B4A4
:10FAF00000FEFDCF8091D8008F7D8093D80080914B
:10FB0000E1008F7E8093E1008091E2008F7E809300
:10FB1000E2008091E20081608093E2008091960192
:10FB2000882311F084E007C08091E30087FF02C0C2
:10FB300083E001C081E08EBB38D18091E10083FF7A
:10FB400021C08091E20083FF1DC08091E100877F8A
:10FB50008093E10082E08EBB109296018091E100DB
:10FB60008E7F8093E1008091E2008E7F8093E2009F
:10FB70008091E20080618093E20042E060E080E0FA
:10FB8000D1DE13D1FF91EF91BF91AF919F918F91F2
:10FB90007F916F915F914F913F912F910F900FBE89
:10FBA0000F901F9018951F93CF93DF9300D0CDB780
:10FBB000DEB7E8E9F1E08091F100819381E0E03A7D
:10FBC000F807C9F759DD8091E80083FFDAC090910A
:10FBD000980180919901853009F465C030F4813035
:10FBE00059F168F0833041F1CCC0883009F49CC0F1
:10FBF000893009F4ABC0863009F0C3C075C09038B5
:10FC000081F0923809F0BDC080919C018F70809383
:10FC1000E9009091EB0095FB992790F91092E9008B
:10FC200001C090E08091E800877F8093E800909386
:10FC3000F1001092F10083C0292F2D7F09F0A1C09F
:10FC4000923009F09EC090919A01911126C02091A6
:10FC50009C012F7009F495C02093E9009091EB006E
:10FC600090FF1BC0833021F48091EB00806213C0B1
:10FC70008091EB0080618093EB0081E090E0022EA8
:10FC800001C0880F0A94EAF78093EA001092EA0014
:10FC90008091EB0088608093EB001092E9008091E6
:10FCA000E800877F4FC091116CC010919A011F77B7
:10FCB0008091E3008078812B8093E3008091E800BD
:10FCC000877F8093E80042DE8091E80080FFFCCFD0
:10FCD0008091E30080688093E300112311F083E0BA
:10FCE00001C082E08EBB4DC09058923008F049C0F0
:10FCF000AE014F5F5F4F60919C0180919A0190919E
:10FD00009B01F4DC009709F43CC02091E800277FB8
:10FD10002093E800BC0189819A816DDD8091E80023
:10FD20008B778093E8002DC0903859F58091E800DA
:10FD3000877F8093E800809196018093F100809105
:10FD4000E8008E778093E80001DE1BC0911119C096
:10FD500090919A019230A8F48091E800877F809377
:10FD6000E80090939601F2DD80919601811104C024
:10FD70008091E30087FF02C084E001C081E08EBB78
:10FD80006FDC8091E80083FF0AC08091E800877FE4
:10FD90008093E8008091EB0080628093EB000F90ED
:10FDA0000F90DF91CF911F9108950895CF938EB357
:10FDB0008823A9F08091E9008F709091EC0090FF6A
:10FDC00002C090E801C090E0C92FC82B1092E90052
:10FDD0008091E80083FDE7DECF70C093E900CF910A
:10FDE0000895F999FECF92BD81BDF89A992780B503
:10FDF0000895262FF999FECF1FBA92BD81BD20BD6F
:10FE00000FB6F894FA9AF99A0FBE01960895F894ED
:02FE1000FFCF22
:10FE1200010000000000000812034C0055004600DB
:10FE22004100200043004400430000001803440046
:10FE3200650061006E002000430061006D006500F6
:10FE42007200610000000403090409023E0002017D
:10FE520000803209040000010202010005240010A2
:10FE6200010424020205240600010705820308009A
:10FE7200FF09040100020A00000007050402100045
:10FE82000507058302100005120110010200000897
:10FE9200EB034A200001010200014C554641434454
:02FEA20043001B
:10FFA000D8CBE9CBFACB06CC0BCC10CC16CC089531
:08FFB0000895089508950895D5
:10FFE000DFCFDFCFDFCFDFCFDFCFDFCFDFCFDFCFA1
:08FFF000DFCFDFCFDFCFDFCF51
:08FFF80000F0000000DFFBDC5B
:040000030000F00009
:00000001FF
